:1000000012C01895189518951895189584C21895CA
:100010001895189518951895189518951895189578
:100020001895189518958FED8DBFC0ECE8EB4E2E06
:10003000DD275D2EEEE7F0E0A0E6B0E0A89584B7FE
:10004000082E877F84BF88E1992781BD91BD8827CD
:100050008D933197E9F766248FEF87BB8FEF88BBCD
:100060008EE081BB8FEF82BB82E083BF80E080BFE8
:1000700089B7826089BF789481E0809374008AEFA9
:1000800080937A00E1E0F0E0ABE791E08DD300915E
:100090007B000A3010F009F005C080917B0080934E
:1000A000640003C081E080936400E2E0F0E0ABE72D
:1000B00091E07AD300917B000A3010F009F005C07E
:1000C00080917B008093650003C081E08093650090
:1000D000E3E0F0E0ABE791E067D300917B000A300A
:1000E00010F009F005C080917B008093660003C08A
:1000F00081E080936600E4E0F0E0ABE791E054D368
:1001000000917B00043681E010F009F080E08F93CD
:1001100000917B00013081E008F480E09F91892309
:10012000882309F405C080917B0080936C0003C094
:1001300081E080936C00A8E716D30091770000302F
:1001400009F017C0A0E30C9104FB81E00EF080E001
:100150008F93A0E30C9105FB81E00EF080E09F916E
:100160008923882309F404C0A7E78C918F5F8C93BF
:100170008BC0013009F037C0A0E30C9104FB81E093
:100180000EF080E08F93A0E30C9105FB81E00EF46C
:1001900080E09F918923882309F409C081E090E0E1
:1001A000A8E78D939C93A7E78C918F5F8C93A0E336
:1001B0000C9104FB81E00EF480E08F93A0E30C919E
:1001C00005FB81E00EF080E09F918923882309F4EC
:1001D00009C08FEF9FEFA8E78D939C93A7E78C91C1
:1001E0008F5F8C9351C0023009F017C0A0E30C91CF
:1001F00004FB81E00EF480E08F93A0E30C9105FBFB
:1002000081E00EF480E09F918923882309F404C0E3
:10021000A7E78C918F5F8C9337C0033009F034C00F
:10022000A0E30C9104FB81E00EF080E08F93A0E34B
:100230000C9105FB81E00EF480E09F9189238823D7
:1002400009F408C08FEF9FEFA8E78D939C9380E09F
:1002500080937700A0E30C9104FB81E00EF480E032
:100260008F93A0E30C9105FB81E00EF080E09F915D
:100270008923882309F408C081E090E0A8E78D93E2
:100280009C9380E080937700A8E70D911C9100304B
:1002900050E0150709F45AC080E080937A00A8E77F
:1002A0000D911C91013050E0150709F02AC0A8E615
:1002B0008C9186FB0EF00FC080916C008150809372
:1002C0006C0000916C00013010F009F003C081E077
:1002D00080936C0015C0A4E7AD90A3E6AA0D8C91A5
:1002E0008F5F8C93A4E7AD90A3E6AA0D0C910A3022
:1002F00008F406C08AE0A4E7AD90A3E6AA0D8C93AB
:1003000025C0A8E68C9186FB0EF00DC0ACE68C9162
:100310008F5F8C9300916C00043608F403C084E670
:1003200080936C0013C0A4E7AD90A3E6AA0D07D29A
:10033000A4E7AD90A3E6AA0D0C910A3F08F406C00D
:1003400080E0A4E7AD90A3E6AA0D8C93A8E68C917B
:1003500087FB0EF0DDC0809168008F778093680086
:1003600000917A000A3F08F031C0AAE78C918F5FB4
:100370008C9300917A000A3F09F028C080916400B4
:1003800080937B00E1E0F0E0ABE791E07BE7FBD11D
:100390008091650080937B00E2E0F0E0ABE791E0C4
:1003A0007BE7F1D18091660080937B00E3E0F0E091
:1003B000ABE791E07BE7E7D180916C0080937B0015
:1003C000E4E0F0E0ABE791E07BE7DDD1A8E68C91DB
:1003D00086FB0EF022C0ABE68C918F5F8C93409130
:1003E0006C0000916B00041708F416C080E0809345
:1003F0006B009398919882B394E0892782BBA2E71F
:10040000A2D1A2E70D911C91043853E0150709F021
:1004100002C0A2E7A8D169D135C081E080936D0008
:1004200000916D00033010F009F016C0ADE6AD90FC
:10043000A3E6AA0D0C91ADE6AD90A3E6AA0D4C91F2
:10044000BAD1ADE6AD90A0E6AA0D4C93ADE68C9185
:100450008F5F8C9308F4E4CF00917400013009F0B1
:1004600004C0939A919892980DC0023009F004C08C
:100470009398919A929806C0033009F003C093981C
:100480009198929A80991AC000917500043608F0EC
:1004900014C0A5E78C918F5F8C9300917500043098
:1004A00009F003C081E0809376000091750002336B
:1004B00009F003C082E0809376002AC080E0809338
:1004C000750000917600013009F00FC080E0809344
:1004D0007600A4E78C918F5F8C93009174000430B8
:1004E00009F003C081E0809374000091760002302F
:1004F00009F00EC080E080937600A8E68C9186FB20
:10050000882780F9809580FBA8E68C9186F98C93EA
:1005100012CEF894FFCF0F921F922F923F924F92DC
:100520005F927F92AF92BF920F931F932F933F934F
:100530004F935F936F937F938F939F93AF93BF93EB
:10054000CF93DF93EF93FF938FB78F9380E88093E0
:100550005200A0E68C918F5F8C930091600004366E
:1005600009F003C080E08093600040916100009139
:100570006000041708F402C0C79801C0C79A4091F0
:10058000620000916000041708F402C0C69801C020
:10059000C69A4091630000916000041708F402C0FD
:1005A000C59801C0C59AA9E6CED0A9E60D911C91C7
:1005B0000A3F50E0150709F007C0A9E6D4D08091A2
:1005C00068008068809368008F918FBFFF91EF91E2
:1005D000DF91CF91BF91AF919F918F917F916F915B
:1005E0005F914F913F912F911F910F91BF90AF90CD
:1005F0007F905F904F903F902F901F900F90189595
:10060000AEE60D911C91033853E0150710F009F088
:1006100001C00AC0AEE60D911C9144E853E0041BF2
:10062000150BAEE60D931C93AEE60D911C910436AE
:1006300050E0150780E010F009F081E08F93AEE6FE
:100640000D911C91043F51E0150781E008F080E016
:100650009F918923882309F402C0A0E784D0AEE6E5
:100660000D911C91043650E0150710F009F00AC0F6
:1006700004E610E0AEE64D915C91041B150BA0E77B
:100680000D931C93AEE60D911C91043F51E01507AC
:1006900081E008F480E08F93AEE60D911C9108355F
:1006A00052E0150781E010F009F080E09F91892366
:1006B000882309F40AC0AEE60D911C9144EF51E085
:1006C000041B150BA0E70D931C93AEE60D911C9136
:1006D000083552E0150710F009F001C005C084E6A6
:1006E00090E0A0E78D939C930895A2E78D919C9153
:1006F000AEE68D939C9384DF8091700080936100BF
:10070000A2E70D911C914CE251E0040F151FAEE6DB
:100710000D931C9375DF8091700080936200A2E7B7
:100720000D911C9148E552E0040F151FAEE60D93A4
:100730001C9366DF809170008093630008958C9114
:1007400081508C930895ED91FC91EF5FFF4FFC93E6
:10075000EE9308953197F1F70895689462F808953B
:10076000E89462F8089582E001C084E099279D939F
:100770008A95E9F70895E199FECFEEBB3196089589
:1007800091E001C092E07B3751F47FB7F894F3DF3A
:100790008D918DBBE29AE19A9A95C9F77FBF772731
:1007A000089591E001C092E0E6DFE09A8DB38D9369
:1007B0009A95D1F70895FF935527F8E0469508F4E8
:0E07C000500F57954795FA95D1F7FF91089580
:00000001FF
